:1000000000008A150A12382FF200030E8301F10056
:100010000A088A01F000040883160317D200831629
:100020000317CD01831203130B1D19288316031721
:10003000CD0A831603174D08013A031D24288A159B
:100040000A1273218A110A128316031752088400B8
:1000500070088A008301710E8300F20E720E09008F
:1000600083160313C3007F08C2007E08C1007D0809
:1000700083160313D30083160313C0007C08C70044
:100080007B08C6007A08C500790883160313D700D9
:1000900083160313C400410883160313D400831688
:1000A0000313420883160313D50083160313430872
:1000B00083160313D6008316031345088316031310
:1000C000D80083160313460883160313D90083163A
:1000D0000313470883160313DA0083160313530828
:1000E00083160313C00083160313540883160313E7
:1000F000C10083160313550883160313C200831629
:100100000313560883160313C30040084104420436
:1001100043040319A92883160313570883160313EE
:10012000C00083160313580883160313C1008316F7
:100130000313590883160313C200831603135A08C6
:1001400083160313C3004008410442044304031D03
:10015000B1280030FD000030FE000030FF0000300C
:10016000CC2B83160313530883160313C000831686
:100170000313540883160313C10083160313550891
:1001800083160313C2008316031356088316031342
:10019000C300430DC401C40DC501C601C701013030
:1001A0004405C000C101C201C301831603135708EF
:1001B00083160313C400831603135808831603130E
:1001C000C50083160313590883160313C60083164C
:1001D00003135A0883160313C700470DC801C80D3F
:1001E000C901CA01CB0101304805C400C501C601DF
:1001F000C7014408C0060030C1060030C206003006
:10020000C3064008C4008316031353088316031360
:10021000C00083160313540883160313C10083160A
:100220000313550883160313C200831603135608DD
:1002300083160313C300420D430DC000C500C60161
:10024000C60DC701C801C101C201C3018230C00788
:10025000FF30031CC107FF30031CC207FF30031C23
:10026000C3074008C5004108C6008316031357089A
:1002700083160313C0008316031358088316031351
:10028000C10083160313590883160313C200831693
:1002900003135A0883160313C300420D430DC00015
:1002A000C700C801C80DC901CA01C101C201C3010B
:1002B0004508C7004608C8000030C81BFF30CA0008
:1002C000C90040084707C00048080318480FC10785
:1002D00049080318490FC2074A0803184A0FC30701
:1002E0004008C5004108C60083160313530883164F
:1002F0000313C00083160313540883160313C100AD
:1003000083160313550883160313C20083160313C1
:10031000560883160313C300C213C301C217400853
:1003200083160313D30083160313410883160313A4
:10033000D40083160313420883160313D50000303C
:10034000D60083160313570883160313C0008316C1
:100350000313580883160313C100831603135908A7
:1003600083160313C200831603135A08831603135C
:10037000C300C213C301C217400883160313D7007A
:1003800083160313410883160313D800831603133F
:10039000420883160313D9000030DA0083160313D2
:1003A000530883160313C0008316031354088316DF
:1003B0000313C700C10083160313550883160313E4
:1003C000C800C20083160313560883160313C9001E
:1003D000C300CA0183160313570883160313C00012
:1003E00083160313580883160313CB00C10083162A
:1003F0000313590883160313CC00C200831603139A
:100400005A0883160313CD00C300CE014B08F90030
:100410004C08FA004D08FB000030FC004708FD00C6
:100420004808FE004908FF0000308A110A16D02053
:100430008A110A1283160313C3007F08C2007E08C4
:10044000C1007D08C00083160313530883160313ED
:10045000C70083160313540883160313C8008316BA
:100460000313550883160313C90083160313560894
:1004700083160313CA00C801C901CA0183160313F6
:10048000570883160313CB008316031358088316EB
:100490000313CF00CC0083160313590883160313EC
:1004A000CD00831603135A0883160313CE00D2011E
:1004B0004F08F9004D08D000FA004E08D100FB00AB
:1004C0000030FC004708FD000030FE000030FF0057
:1004D00000308A110A16D0208A110A1283160313DB
:1004E000CD00CA007F08CC00C9007E08CB00C80040
:1004F0007D08C700CE014B08C0074C0803184C0FFD
:10050000C1074D0803184D0FC2074E0803184E0FC0
:10051000C30783160313570883160313C7008316F4
:100520000313580883160313C800831603135908CE
:1005300083160313C900831603135A088316031383
:10054000CA00C801C901CA018316031353088316E0
:100550000313CB0083160313540883160313CC0034
:1005600083160313550883160313D000CD0083169A
:100570000313560883160313D100CE00D2014C0892
:10058000CF00F9005008FA005108FB000030FC00D1
:100590004708FD000030FE000030FF0000308A11E7
:1005A0000A16D0208A110A1283160313CD00CA003E
:1005B0007F08CC00C9007E08C8007D08C700CE01B6
:1005C0004808CB00C00703184C0FC1074D0803189B
:1005D0004D0FC2074E0803184E0FC307C7018030E6
:1005E0004305CA004A080319052B8030C0070318C9
:1005F000C10A0319C20A0319C30A4108C00042080C
:10060000C1004308C200C3011C2B403083160313F2
:10061000C0070318C10A0319C20A0319C30A400D0F
:10062000410DC000420DC100430DC200C301C30D06
:10063000FF30C507031CC60383160313C213460805
:10064000803E7F3E031D262B00304502031C552BA8
:100650008316031344080319332BC701C801C901CA
:100660008030CA00392B83160313C701C801C901A2
:10067000CA0183160313C9177F30CA0447088316BB
:100680000313D30083160313480883160313D400FF
:1006900083160313490883160313D5008316031327
:1006A0004A0883160313D600AD2B031483160313D5
:1006B000C61F0310031C632B83160313D301D4013D
:1006C000D501D601AD2B0030831603134404031962
:1006D0006F2BC401C701C8018030C900752B831678
:1006E0000313C401C701C801C901831603134508D8
:1006F000CA004608CB000030CB1BFF30CD00CC0039
:100700004B0C4A0CCF00CE01CE0CC601C501003007
:10071000C4040030C7044E08C8044F08C904440884
:10072000C0044708C1044808C2044908C30440087B
:1007300083160313D3008316031341088316031390
:10074000D40083160313420883160313D5008316BF
:100750000313430883160313D600831603135308A9
:1007600083160313C0008316031354088316031360
:10077000C10083160313550883160313C2008316A2
:100780000313560883160313C3004008FD004108F5
:10079000FE004208FF004308080083120313A30071
:1007A0007F08A2007E08A1007D0883120313BB000E
:1007B00083120313A0007C08A7007B08A6007A0818
:1007C000A500790883120313BF0083120313A4004A
:1007D000A801A901AA01AB01210883120313BC00DF
:1007E00083120313220883120313BD008312031321
:1007F000230883120313BE008312031325088312F8
:100800000313C00083120313260883120313C100CD
:1008100083120313270883120313C20083120313E6
:100820003B0883120313A000831203133C088312B6
:100830000313A100831203133D0883120313A200C4
:10084000831203133E0883120313A300200821041C
:1008500022042304031D4C2C831203133F0883122C
:100860000313A00083120313400883120313A10093
:1008700083120313410883120313A200831203138C
:10088000420883120313A3002008FD002108FE0084
:100890002208FF002308F52E831203133F0883125A
:1008A0000313A00083120313400883120313A10053
:1008B00083120313410883120313A200831203134C
:1008C000420883120313A3002008210422042304F6
:1008D000031D8A2C831203133B0883120313A00009
:1008E000831203133C0883120313A1008312031322
:1008F0003D0883120313A200831203133E088312E0
:100900000313A3002008FD002108FE002208FF00B9
:100910002308F52E831203133B0883120313A00050
:10092000831203133C0883120313A10083120313E1
:100930003D0883120313A200831203133E0883129F
:100940000313A300220D230DA000A400A501A50DF3
:10095000A601A701A101A201A3012008A400003063
:10096000A500831203133F0883120313A000831210
:100970000313400883120313A100831203134108D9
:1009800083120313A200831203134208831203137A
:10099000A300220D230DA000A600A701A70DAC0106
:1009A000AD01A101A201A3010030A7001930260763
:1009B000A000A101A10D2708A1072108803EAE00DB
:1009C0002508803E2E02031DE72C24082002031870
:1009D000092D831203133B0883120313A000831213
:1009E00003133C0883120313A100831203133D0871
:1009F00083120313AC00831203133E088312031304
:100A0000AD002008FD002108FE002C08FF002D0885
:100A1000F52E1930831203132407A000A101A10DA4
:100A20002508A1072108803EAE002708803E2E023F
:100A3000031D1C2D2608200203183E2D83120313CC
:100A40003F0883120313A00083120313400883128C
:100A50000313A10083120313410883120313AC0094
:100A600083120313420883120313AD002008FD0014
:100A70002108FE002C08FF002D08F52E8312031319
:100A80003B0883120313A000831203133C08831254
:100A90000313A100831203133D0883120313AC0058
:100AA000831203133E0883120313AD00AC13AD0190
:100AB000AC17831203133F0883120313AE00831293
:100AC0000313400883120313AF008312031341087A
:100AD00083120313B000831203134208831203131B
:100AE000B100B013B101B017831203133B08831296
:100AF0000313B200831203133C0883120313B300E1
:100B0000831203133D0883120313B40083120313EB
:100B10003E0883120313B500350DB601B60DB701BB
:100B2000B801B901361C9F2DA009A109AC09AD0976
:100B3000A00A0319A10A0319AC0A0319AD0A83120A
:100B400003133F0883120313B200831203134008F8
:100B500083120313B3008312031341088312031398
:100B6000B40083120313420883120313B500350D3A
:100B7000B601B60DB701B801B901361CCA2DAE09D0
:100B8000AF09B009B109AE0A0319AF0A0319B00AD7
:100B90000319B10A831203132708803EBA002508FF
:100BA000803E3A02031DD62D240826020318FD2D8F
:100BB0008312031326082402B2002708031C270A05
:100BC0002502B3003208B21BF22D003C0319FC2DA4
:100BD00083120313B10CB00CAF0CAE0C013E031C1E
:100BE000E82DFC2D031083120313AE0DAF0DB00DD5
:100BF000B10D013E031CF32D272E8312031324088D
:100C00002602B2002508031C250A2702B300320879
:100C1000B21B172E003C0319212E83120313AD0CB7
:100C2000AC0CA10CA00C013E031C0D2E212E0310B8
:100C300083120313A00DA10DAC0DAD0D013E031CDD
:100C4000182E831203132608A4002708A500831278
:100C500003132E08A0072F0803182F0FA107300831
:100C60000318300FAC0731080318310FAD07200807
:100C7000A6002108A7002C08AE002D08AF00031421
:100C8000AF1F0310031C552EA009A109AC09AD0923
:100C9000A00A0319A10A0319AC0A0319AD0AA80195
:100CA000A901AA018030AB00652E8312031320082E
:100CB00021042C042D04031D652E0030FD0000309E
:100CC000FE000030FF000030F52E003083120313C9
:100CD0002D02031D752E80302C02031D752E003051
:100CE0002102031D752E003020020318832E0310ED
:100CF00083120313A00DA10DAC0DAD0DFF30A407A1
:100D0000031CA503652E83120313A6012D08AF0053
:100D100003199F2E201C942E0230A0070318A10A4D
:100D20000319AC0A0319AD0A031083120313AD0CA7
:100D3000AC0CA10CA00CA40A0319A50A832E8312E3
:100D40000313AC132408A6002508A7000030A71B36
:100D5000FF30AF00AE00270C260CB100B001B00C84
:100D6000A501A4010030A8040030A9043008AA0499
:100D70003108AB042808A0042908A1042A08AC04FF
:100D80002B08AD04200883120313BB008312031346
:100D9000210883120313BC00831203132C0883124F
:100DA0000313BD00831203132D0883120313BE0027
:100DB0003B0883120313A000831203133C08831221
:100DC0000313A100831203133D0883120313A4002D
:100DD000831203133E0883120313A5002008FD00AD
:100DE0002108FE002408FF002508080083120317CD
:100DF00093007F0892007E0891007D0883120317FC
:100E000099008312031790007C0897007B089600D6
:100E10007A0895007908831203179D00831203173F
:100E200094001108831203179A0083120317120803
:100E3000831203179B0083120317130883120317EF
:100E40009C00831203171508831203179E00831258
:100E500003171608831203179F008312031717083E
:100E600083120317A00083120317190883120317B4
:100E70009000831203171A0883120317910083123C
:100E800003171B08831203179200831203171C0811
:100E90008312031793000314931F0310031CB52F31
:100EA000831203171D088312031790008312031780
:100EB0001E08831203179100831203171F08831261
:100EC000031792008312031720088312031793005D
:100ED0000314931F0310031CB52F831203171D085F
:100EE000831203179000831203171E08831203173F
:100EF0009100831203171F088312031792008312B5
:100F0000031720088312031793008312031719088D
:100F1000831203179400831203171A08831203170E
:100F20009500831203171B08831203179600831280
:100F300003171C088312031797001308803E9800BC
:100F40001708803E1802031DAF2F16081202031D5A
:100F5000AF2F15081102031DAF2F1408100203183C
:100F6000B32F0130FC2F0030FC2F83120317190818
:100F7000831203179000831203171A0883120317B2
:100F80009100831203171B08831203179200831228
:100F900003171C08831203179300831203171D08FD
:100FA000831203179400831203171E08831203177A
:100FB0009500831203171F088312031796008312EC
:100FC000031720088312031797001308803E980028
:100FD0001708803E1802031DF72F16081202031D82
:100FE000F72F15081102031DF72F1408100203181C
:0C0FF000FB2F0130FC2F00300800003403
:1010000083160313860183160317CF01013083165D
:101010000317D10083120313DB0183120313D801DA
:101020000830831203135802031826285808A13EDB
:10103000D90001300318013EDA00590884008313F7
:101040005A188317B7308000D80A10288316031760
:10105000CE0183160317D001692108008312031300
:10106000D6000130D7005608003C03193D288312F2
:101070000313D70D013E031C3728831203135709AE
:10108000D60083160317CE05080083120313D4007D
:101090000130D5005408003C03195428831203136F
:1010A000D50D013E031C4E288312031355088316E9
:1010B0000317CE04080083160317CE00080083121E
:1010C0000313D1007F08D0007E087D08D2005008AD
:1010D000A13ED00051080318510F013ED100520823
:1010E000D3005008840083135118831753088000DD
:1010F000080083120313CC007F08CB007E08CE00CB
:101100007D08CD00FF004E089C2083120313CE0003
:101110007F08CD004B08A13ECB004C0803184C0FB4
:10112000013ECC004D08CF004B08840083134C18BF
:1011300083174F088000080083120313C6007F083E
:10114000C5000314C61F0310031801294508FF003A
:1011500046088A110A1600248A150A1283120313FC
:10116000CA007F08C9007E08C8007D08C700F900D2
:101170004808FA004908FB004A08FC00CD30FD0091
:10118000CC30FE004C30FF003F308A110A12302074
:101190008A150A1283120313CA007F08C9007E0849
:1011A000C8007D08C7000030F9000030FA00903018
:1011B000FB004230FC004708FD004808FE004908DB
:1011C000FF004A088A110A12CD238A150A128312D7
:1011D0000313CA007F08C9007E08C8007D08C70045
:1011E000FD004808FE004908FF004A088A110A1657
:1011F00030238A150A1283120313C8007F08C70020
:101200005C2983120313450983120313DC00831244
:101210000313460983120313DD00DC0A0319DD0AF8
:101220005C08FF005D088A110A1600248A150A125C
:1012300083120313CA007F08C9007E08C6007D0818
:10124000C500F9004608FA004908FB004A08FC00FE
:10125000CD30FD00CC30FE004C30FF003F308A1115
:101260000A1230208A150A1283120313E1007F0844
:10127000E0007E08DF007D08DE005E08FD005F08FC
:10128000FE006008FF0061088A110A1630238A15E3
:101290000A1283120313E3007F08E2006208483C4D
:1012A00083120313C700831203136308031C630A2A
:1012B000003C83120313C80083120313C7090314ED
:1012C0004808031C480A003CC8004708FF004808BB
:1012D00008000530831603138100831203130B11DA
:1012E0008B1681010800831203130B118312031361
:1012F0005B08031D8E2983160317510883160317F5
:101300004E05831203138600EA30810001308312F8
:101310000313DB0083160317D000E42983120313A1
:101320005B08013A031DAD29831603174F08A13E40
:1013300083120313C30001300318013EC4004308A5
:101340008400831344188317000883120313810059
:10135000023083120313DB00E429831203135B08BA
:10136000023A031DE1298312031386018316031732
:101370004F08A13E83120313C30001300318013E3E
:10138000C400430884008313441883170008523CA8
:1013900083120313810083120313DB0103108316EE
:1013A0000317D10D83160317CF0A003083160317D6
:1013B0005104031DE4290130D10083160317CF0126
:1013C000E42983120313DB01080083160313B6001C
:1013D0007F08B500831603175008013A031DA82A99
:1013E000D001831603174F0883160313B70002308A
:1013F000FF0037088A110A1628248A150A12831654
:101400000313B800213EB90001300318013EBA00B1
:101410003908840083133A1883170008BB00840A34
:101420000008BC003808313EB80001300318013E06
:10143000B900380884008313391883170008BA00EC
:10144000840A0008BD003A08831603133E0783167A
:101450000313B800831603133F0883160313B90060
:101460003D0803183D0FB9073808FD003908FE0094
:101470003B08FF003C088A150A1235258A150A1216
:1014800083160313B9007F08B8003708993EBA00E5
:1014900001300318013EBB003A08840083133B1857
:1014A00083170008BC00BA00BB01BA1BBB033A0893
:1014B000B8073B0803183B0FB9073808FF00390885
:1014C0008A150A129C208A150A1283160313B90082
:1014D0007F08B800BA003708A13EB80001300318F1
:1014E000013EB900380884008313391883173A087D
:1014F00080003708031DA82A350883160313BE078A
:101500008316031336080318360A03198A2A83162A
:101510000313BF07031483160313BF1F0310031C19
:10152000952A6730BE000130BF006830FD000130F1
:10153000FE00831603133E08FF003F088A110A16B7
:1015400062218A150A1283160313BF007F08BE00AA
:10155000080083160313A1007F08A0007E08A300E3
:101560007D08A2007C08A5007B08A4007A08A700DB
:101570007908A6007808A9007708A8007608AB00CB
:101580007508AA007408AC00AD010130AE00093046
:10159000831603132E020318BC2B2E087F3EAF00C8
:1015A00014300318013EB0002F08FE003008FF0081
:1015B00080308A110A1668228A150A1283160313CC
:1015C000B10031080319B82B01302E05AF00013AE4
:1015D000031D422B2E08AF00B001FF30AF07031CE4
:1015E000B0030310B01B0314300C2F0CB200AF007B
:1015F0003103B2000230FF0032088A110A16282493
:101600008A150A1283160313B000213EB20001307E
:101610000318013EB3003208840083133318831784
:1016200020088000840A2108800084033008313EAD
:10163000B00001300318013EB200B4012408FD00DF
:101640002508FE002F08B300FF0000308A110A169B
:10165000C2238A150A1283160313B4007F08B3004D
:101660002A08B3072B0803182B0FB407300884008F
:1016700083133218831733088000840A34088000EB
:101680008403A52B0310831603132E0CB000300324
:10169000AF003103B0000230FF0030088A110A1693
:1016A00028248A150A1283160313B200213EB300C0
:1016B00001300318013EB40033088400831334184A
:1016C000831722088000840A2308800084033208DC
:1016D000313EB20001300318013EB3002608FD0080
:1016E0002708FE002F08B400FF0000308A110A16F8
:1016F000C2238A150A1283160313B4007F08AF00B1
:101700002808AF0729080318290FB4072A08AF07CC
:101710002B0803182B0FB4073208840083133318E7
:1017200083172F088000840A34088000840330085F
:10173000993EB00001300318013EAF00300884002C
:1017400083132F1883172C08800083160313B1030B
:101750000130AF003108003C0319B42B831603138A
:10176000AF0D013E031CAE2B831603132F08AD04EF
:1017700083160313AE0AC72A831603132D088A158E
:101780000A125B208A150A1283160313BE01BF01D9
:10179000080000340034003400347F34F7348E34D1
:1017A0003C344134F2340E343D3446345E345634E5
:1017B0003D343C34DC348E343D34D8347E34B23461
:1017C0003D34D3341334D6343D34FB349634F934B9
:1017D0003D34953482340E343E3430342F3420344A
:1017E0003E344E34D13431343E34B2346334433435
:1017F0003E345C34E63454343E344B34593466342D
:101800003E34E034B93477343E340E348434843496
:101810003E34B03420348D343E348534B134953484
:101820003E34DF3437349E343E341C34B134A63475
:101830003E343F341D34AF343E3446347C34B73408
:101840003E34E234CC34BF343E34C3340D34C83477
:101850003E343A344034D0343E34A6346134D83443
:101860003E3408347234E0343E3461347134E83448
:101870003E345F345E34F0343E3404343934F8346A
:101880003E340034003400343F34A934D9340334B6
:101890003F34D634A83407343F3487346D340B34A6
:1018A0003F34133427340F343F342434D6341234C5
:1018B0003F346834793416343F34E03410341A3409
:1018C0003F34E5349B341D343F341E341B34213403
:1018D0003F34E3348D3424343F348C34F3342734B0
:1018E0003F341B344C342B343F348D3497342E34F6
:1018F0003F343D34D53431343F3429340534353424
:101900003F34AB34263438343F34C13439343B347B
:101910003F346C343E343E343F34AD34343441349F
:101920003F3433341B3444343F344D34F334463481
:101930003F340634BB3449343F34AC3473344C3414
:101940003F34EF341B344F343F34D034B33451344C
:101950003F34F7343B3454343F341434B3345634C6
:101960003F34CE34193459343F347E346F345B34D1
:101970003F342434B4345D343F341934E7345F34B5
:101980003F340334093462343F343B341934643413
:101990003F341A34173466343F34EF340334683438
:1019A0003F346A34DE3469343F34E334A5346B3475
:1019B0003F34AB345B346D343F341934FF346E3410
:1019C0003F3486348F3470343F3499340D3472345C
:1019D0003F34AB34783473343F341434D0347434FB
:1019E0003F342334153476343F343034473477343D
:1019F0003F349534653478343F345034703479341E
:101A00003F340A3468347A343F341B344C347B34EA
:101A10003F3482341C347C343F344034D9347C34F9
:101A20003F34563482347D343F34C23417347E34EC
:101A30003F34DD3498347E343F344F3406347F34C1
:101A40003F34183460347F343F343734A6347F3425
:101A50003F340634D8347F343F342B34F6347F346B
:101A60003F340034003480343F3483120317D200F3
:101A70007F08D1007E08D4007D08D3000130D50056
:101A8000D6010314D41F031003184A2D0130D700C8
:101A9000D801542DFF3083120317D700D800D30983
:101AA000D409D30A0319D40A6830FD000130FE00BE
:101AB000831203175308FF0054088A110A16622183
:101AC0008A150A1283120317D4007F08D300540822
:101AD000803E803E031D6E2D5B305302031C852D1E
:101AE000831203175408803E803E031D792DB530C4
:101AF00053020318852D831203175308B43CD300F7
:101B00005408031C540A003CD400831203175408E1
:101B1000803E803E031D8E2DB5305302031CA42D44
:101B2000831203175408803E7F3E031D992D0F300A
:101B300053020318A42D4C3083120317D307031C40
:101B4000D403FF30D500D600831203175408803E1B
:101B50007F3E031DAD2D0F305302031CC72D831292
:101B600003175408803E7F3E031DB82D6930530291
:101B70000318C72D831203175308683CD300540879
:101B8000031C540A013CD400FF30D500D600831258
:101B900003175308FD005408FE000430FF00003016
:101BA0008A110A16C2238A150A1283120317D40057
:101BB0007F08D300C93ED30054080318540F0B3ECE
:101BC000D4005308FE005408FF0080308A110A1622
:101BD0007B228A150A1283120317DC007F08DB00C0
:101BE0007E08DA007D08D9005108FF0052088A11EA
:101BF0000A1600248A150A1283120317D4007F08DC
:101C0000D3007E08D2007D08D1005908F9005A0897
:101C1000FA005B08FB005C08FC005108FD0052085C
:101C2000FE005308FF0054088A110A1230208A155A
:101C30000A1283120317D4007F08D3007E08D20053
:101C40007D08D100FD005208FE005308FF00540833
:101C50008A110A1630238A150A1283120317DE002E
:101C60007F08DD00831203175508FD005608FE00AB
:101C70005708FF0058088A110A16C2238A150A124B
:101C800083120317D2007F08D100831203175D0867
:101C9000FD005E08FE00831203175108FF00520882
:101CA0008A110A16C2238A150A1283120317D20058
:101CB0007F08D100FF005208080083120317E200DA
:101CC0007F08E1007E08E0007D08DF008312031733
:101CD000E70083120317600883120317E8008312DA
:101CE0000317610883120317E900831203176208C0
:101CF00083120317EA00670883120317DF008312B9
:101D00000317680883120317E0008312031769089A
:101D100083120317E100831203176A088312031763
:101D2000E2005F086004610462040319B72E8312A5
:101D30000317670883120317DF008312031768086D
:101D400083120317E0008312031769088312031735
:101D5000E100831203176A0883120317E200620D81
:101D6000E301E30DE401E501E601631CBF2E003051
:101D7000FD000030FE000030FF000030372F8312DE
:101D80000317670883120317DF008312031768081D
:101D900083120317E00083120317690883120317E5
:101DA000E100831203176A0883120317E200610D32
:101DB000620DDF00E300E401E40DE501E601E0016E
:101DC000E101E2016A30DF07FF30031CE007FF306A
:101DD000031CE107FF30031CE2075F08E300600813
:101DE000E40083120317670883120317DF008312CE
:101DF0000317680883120317E000831203176908AA
:101E000083120317E100831203176A088312031772
:101E1000E200E113E201E117E309E409E30A03192F
:101E2000E40A6308E31B242F003C03192E2F031040
:101E300083120317E21B0314E20CE10CE00CDF0C2D
:101E4000013E031C172F2E2F031083120317DF0DE3
:101E5000E00DE10DE20D013E031C252F8312031757
:101E60005F08FD006008FE006108FF0062080800CE
:101E70004530FE001430FF0080308A110A16B62269
:101E80008A150A1283120313E5007F08E400473025
:101E9000E6001430E700831203136408E8006508C5
:101EA000E900FF30E407031CE5036808690403192F
:101EB000C82F04306607E800E901E90D6708E90763
:101EC0006808FE006908FF0080308A110A16B622F1
:101ED0008A150A1283120313EB007F08EA006608D2
:101EE000FE006708FF0080308A110A16B6228A15A4
:101EF0000A1283120313ED00E9007F08EC00E800EA
:101F000002306607E800E901E90D6708E90768089B
:101F1000FE006908FF0080308A110A16B6228A1571
:101F20000A1283120313E900EF007F08E800EE00B5
:101F3000831203136A08EE006B08EF00FF30EA0714
:101F4000031CEB036E086F040319C12F6C08FE001D
:101F50006D08FF0080308A110A1668228A150A125D
:101F600083120313EE006808840083136918831733
:101F70006E088000EC0A0319ED0AE80A0319E90A61
:101F8000982F063083120313E6070318E70A4B2F36
:101F90008A150A12CC2F08008A150A1200208A1509
:101FA0000A120030F4000030F5000030F600003076
:101FB000F7000030F8005A30F9000030FA005A30CB
:101FC000FB000030FC001E30FD000030FE0014302D
:101FD000FF0000308A150A12A9228A150A128312FC
:101FE00003138B170430FF0000308A150A12E52115
:081FF0008A150A12F22F080005
:1020000083120317C4007F08C3007E08C2007D0846
:10201000C100420443044404031D16280030FD009F
:102020000030FE000030FF000030CF2896308312D1
:102030000317C500C601831203174408FF390319AB
:102040002A280310C40CC30CC20CC10CC50A031906
:10205000C60A1B28831203174508C7004608C80094
:1020600000304402031D3E2880304302031D3E28F9
:1020700000304202031D3E2800304102031861284F
:10208000031083120317C10DC20DC30DC40DFF3021
:10209000C507031CC60300304402031D59288030C5
:1020A0004302031D592800304202031D5928003005
:1020B0004102031C4028831203174508C700460845
:1020C000C800831203174208C6007F304305C900C9
:1020D000CA014108C500FF3A031D81284608FF3A9E
:1020E000031D812849087F3A031D81284A08003AC8
:1020F000031D8128C101C201C301C401C70A03191C
:10210000C80A83120317C3134708C5004808C6004E
:102110000030C61BFF30CA00C900460C450CCC007D
:10212000CB01CB0CC801C7010030C1040030C20490
:102130004B08C3044C08C404410883120317CD00A4
:1021400083120317420883120317CE00831203176A
:10215000430883120317CF00831203174408831226
:102160000317D0004D0883120317C1008312031711
:102170004E0883120317C200831203174F088312FD
:102180000317C30083120317500883120317C400F8
:102190004108FD004208FE004308FF004408080013
:1021A00083160313DE007F08DD007E08DC007D0857
:1021B000DB007C08E2007B08E1007A08E000790897
:1021C000DF00E301E401E501E6010830E7008316E2
:1021D00003135B1CF9285F08E30760080318600F0E
:1021E000E40761080318610FE50762080318620F2E
:1021F000E607831603135C1C11296108EB006008D5
:10220000EA00E8010030E3075F08E9000318690FFE
:10221000E4076A0803186A0FE5076B0803186B0FD9
:10222000E607831603135D1C29296008EB005F088D
:10223000EA00E901E8010030E30700300318690F04
:10224000E4076A0803186A0FE5076B0803186B0FA9
:10225000E607831603135E1C40295F08EB00EA01C2
:10226000E901E8010030E30700300318690FE407D3
:102270006A0803186A0FE5076B0803186B0FE60777
:10228000831603135B08E8005C08E9005D08EA00B8
:102290005E08EB0003106B0CDE006A0CDD00690CBD
:1022A000DC00680CDB000310DF0DE00DE10DE20D3A
:1022B000E70BE7286308FD006408FE006508FF00DF
:1022C0006608080083160317B2007F08B1007E0875
:1022D000B4007D08B3000314B21F0310031CB4291B
:1022E0000314B41F0310031C97293109B5003209E8
:1022F000B600B50A0319B60A3309B7003409B800A5
:10230000B70A0319B80A3708FD003808FE00350877
:10231000FF0036088A110A167F238A110A168316CF
:102320000317B6007F08B500FF003608EB298316B7
:1023300003173109B5003209B600B50A0319B60A08
:102340003308FD003408FE003508FF0036088A1106
:102350000A167F238A110A1683160317B6007F0810
:10236000B500FF003608EB29031483160317B41FCA
:102370000310031CD6293309B5003409B600B50A89
:102380000319B60A3508FD003608FE003108FF00C3
:1023900032088A110A167F238A110A168316031738
:1023A000B6007F08B500FF003608EB298316031737
:1023B0003308FD003408FE003108FF0032088A119E
:1023C0000A167F238A110A1683160317B2007F08A4
:1023D000B100FF003208080083160317AC007F0825
:1023E000AB007E08AA007D08A9002A042B042C0457
:1023F000031D022A0030FD000030FE000030FF0007
:102400000030672A0030F9000030FA000030FB008D
:102410000030FC00831603172908FD002A08FE007F
:102420002B08FF002C088A110A12F6268A110A16B8
:1024300083160317AD002D0803194A2AB000AD001A
:10244000AE00AF002D08FD002E08FE002F08FF0093
:1024500030088A150A125D268A110A168316031798
:10246000B0007F08AF007E08AE007D08AD00AD096A
:10247000AE09AF09B009AD0A0319AE0A0319AF0AD4
:102480000319B00A2D08FD002E08FE002F08FF00DA
:102490003008672A831603172908FD002A08FE0062
:1024A0002B08FF002C088A150A125D268A110A16CD
:1024B00083160317AC007F08AB007E08AA007D08D6
:1024C000A900FD002A08FE002B08FF002C080800C8
:1024D000003A03196F2A803A0319762A00347E08DD
:1024E000840083137F188317000808007F088A0080
:1024F0007E0882000800003A0319852A803A0319F1
:10250000952AFD01FE01FF0100347E08840083133B
:102510007F1883170008FD00840A0008FE00840A63
:102520000008FF00840A000808008A110A167622B3
:10253000FD00FE0FFF03FF0A8A110A167622FC0037
:10254000FE0FFF03FF0A8A110A167622FB00FE0F18
:10255000FF03FF0A8A110A167622FA007D08FD00A1
:102560007C08FE007B08FF007A080800003A031987
:10257000BE2A803A0319C82AFF0100347E0884006D
:1025800083137F1883170008FF00840A00080800DF
:102590008A110A167622FD00FE0FFF03FF0A8A1138
:1025A0000A167622FC007D08FF007C0808008316CE
:1025B0000317BC007F08BB007E08BA007D08B90085
:1025C0000314BC1F0310031C122B3909BD003A0968
:1025D000BE003B09BF003C09C000BD0A0319BE0A8A
:1025E0000319BF0A0319C00A3D08FD003E08FE009A
:1025F0003F08FF0040088A110A1600208A110A16B7
:1026000083160317C0007F08BF007E08BE007D0848
:10261000BD00C0003D08FD003E08FE003F08FF0071
:1026200040082F2B831603173908FD003A08FE00D7
:102630003B08FF003C088A110A1600208A110A167E
:1026400083160317BC007F08BB007E08BA007D0814
:10265000B900FD003A08FE003B08FF003C080800F6
:1026600083160313EF007F08EE007E08ED007D085F
:10267000EC00FD006D08FE006E08FF006F088A1177
:102680000A16EC218A110A1683160313EF007F083D
:10269000EE007E08ED007D08EC006F08803E803E75
:1026A000031D5C2B00306E02031D5C2B7F306D021E
:1026B000031D5C2BFF306C02031C622BFF30FF00FC
:1026C0007F307E2B831603136F08803E813E031DEF
:1026D000732BFF306E02031D732B80306D02031DC0
:1026E000732B01306C020318792B0030FF0080300F
:1026F0007E2B831603136C08FF006D0808008316F9
:102700000317C8007F08C7007E08CA007D08C900FB
:102710004A04031D8F2BFF30FF00FF30C12B013017
:1027200083160317CB008316031749084A08CC0009
:10273000CC1B9F2B0310C90DCA0DCB0A932B003065
:10274000831603174B040319BC2B4A084802031DC8
:10275000AB2B49084702031CB52B83160317490806
:10276000C7024A08031C4A0FC80203108316031746
:10277000CA0CC90CCB039F2B831603174708FF0015
:10278000480808008316031791007F0890007E0810
:1027900093007D08920094019501083096008316FD
:1027A0000317101CD92B1208940713080318130FD2
:1027B000950783160317100897001108980000303A
:1027C000981BFF30181CEC2B97010030940712085F
:1027D00098000318180F9507831603171008970021
:1027E000110898000310180C9100170C90000310AA
:1027F000920D930D960BCF2B1408FF0015080800BF
:1028000083160317C400C2007F08C100C300003054
:10281000C41BFF30C600C5004308FD004408FE008D
:102820004508FF0046088A110A16D7228A110A169F
:1028300083160317C4007F08C3007E08C2007D080A
:10284000C100FD004208FE004308FF0044080800E4
:1028500083120317EB007F08EC00ED010830EE0057
:10286000831203176B1C362C6C08ED0783120317B9
:102870006B08EF0003106F0CEB0003106C0DEF0002
:10288000EC00EE0B302C6D080800043400345F348B
:10289000143421340134103400346F34143431349E
:1028A0000134103400348834143499340134083439
:1028B0000034FD340734D33401340134003400349F
:1028C0000034003400340034003400340034003468
:1028D0000034003400340034003400340034003458
:1028E0000034003400340034003400340034003448
:1028F0000034003400340034003400340034003438
:102900000134023403340434053406340734083403
:102910000034003400340034003400340034003417
:00000001FF
